:020000020000FC
:1000000069CD0000000000001FC0A4C18DC0000029
:10001000000097C00000000000000000020304067A
:10002000080C10182030406080000406080C1018DE
:100030002030406080A0C0000003070F1F000505AE
:100040000D050305030302004FB662FD0CC05520E9
:1000500041F00994C52DC095089483FDC795C4BD92
:1000600064604FBE1895C0916400089483FDC795E5
:10007000C4BD6B7FC0916400CF3F09F41EC070FF08
:100080001AC082FD05C04FBEAC98929894981895FE
:1000900076FD0EC064FD0CC0C091B100C0FD959806
:1000A000C1FDAD98C2FD9398CAEFC095CA95F1F70E
:1000B000AC98929894984FBE189524BCCC27C064F5
:1000C000C8BF6460F8CFC6CF70FFC4CF64FDC2CF95
:1000D000AC9AC0CF70FFBECF64FDBCCF929ABACFAE
:1000E00070FFB8CF64FDB6CF949AB4CF959A70FFE5
:1000F000B1CF64FDAFCFC7E0CA95F1F7AC9AAACFF4
:10010000AD9A70FFA7CF64FDA5CFC7E0CA95F1F700
:10011000929AA0CF939A70FF9DCF64FD9BCFC7E0CA
:10012000CA95F1F7949A96CF4FB6C9B7CF7EC9BF9B
:100130006E7FCCB5CE0DDDB5DF1DDBBDCABD4FBEBC
:1001400018953FB68F7EA9B7A072A2118061A9B79A
:10015000AF7DA9BFA9B7AE7FA9BF7894A091680071
:10016000AA2341F085FD2FC0A0916800AA95A09315
:10017000680029C040E050E085FD15C0A6B396FD9B
:10018000A095A0FD4FEFAEB5A06496FDAF7BAEBDD0
:10019000AA27A062A8BF8D7FA6B396FDA095A0FD5B
:1001A0005FEF451739F7A8E161FDA093680085FD71
:1001B00003C0A8E1A09368004093960081604423A7
:1001C00011F02092990085FD0EC0A0916900AA232C
:1001D00031F0A0916900AA95A093690004C08061E4
:1001E000AA27A062A8BF80FF3DC0A09196004A2F19
:1001F00061FF8E7F85FD18C0403F08F040EFA42FBF
:10020000A295AF704A0F5091B600533069F0A69591
:10021000A69550FD01C0A69552FD03C0A41B4A2F10
:1002200003C04A0F08F44FEFA0919F004A1708F44B
:100230004A2F40936100A72FA670A1F073FD12C052
:10024000A0917000AA0FAA0F50919E005695569546
:10025000541708F0452F4A0F4093610018F4AFEF90
:10026000A0936100A0916100A0936300409163009E
:10027000A0919B004A1708F04A2F542EA091A0008D
:10028000AA2309F422C0542F5A1B10F4A42F50E0C3
:10029000BA2E8894AA1FAA2EA091A200A095AA22E5
:1002A000A50E58F0A091A100A21509F0AA95AA0EDA
:1002B000A093A10048F04A2D08C0A091A100BA1651
:1002C00008F0A395A093A1004FEF409364007F7BBB
:1002D000485F08F07064A0916000A395A09360004F
:1002E00059F0F894A9B7A160A9BF84FF03C0A9B7CA
:1002F000A062A9BF3FBE1895A0917400A395A093DA
:10030000740041E050916800552329F085FF03C037
:100310005A9550936800A0919600A13018F0209251
:1003200099000DC020929A002092A300A0919900FC
:10033000AF5FA093990018F0AFEFA0939900F894E5
:10034000A9B7A160A9BF84FF03C0A9B7A062A9BFD4
:100350003FBE18953FB646B557B58F7EA9B7A07278
:10036000A2118061A9B7AF7DA9BFA9B7AE7FA9BF10
:10037000789481FD25C0AEB5AF7B96FDA064AEBD7F
:100380008260A6B396FDA095A0FF05C040936500CE
:100390005093660041C1AEB5A06496FDAF7BAEBD83
:1003A000AA27A062A8BF8D7F85FF01C028C140E0B9
:1003B000A6B396FDA095A0FD22C14093960011C161
:1003C000AEB5A06496FDAF7BAEBD8D7F61FF72C000
:1003D000AEB5AF7B96FDA064AEBDAA27A062A8BF54
:1003E00082604093910050939200A0908F004A1930
:1003F000B09090005B09BB24A22C4C38520518F435
:100400002092950049C0A091D400AA2359F1483CFC
:10041000520528F4A0E1BA2EAAE0AA2E23C048363D
:10042000A1E05A0728F4A8E0BA2EAFE0AA2E1AC01D
:10043000403DA2E05A0728F4A4E0BA2EAEE1AA2E6D
:1004400011C0403AA5E05A0728F4A2E0BA2EACE366
:10045000AA2E08C04839A8E05A0720F4A1E0BA2E15
:10046000A8E7AA2EC42EA0919300CA1AD52EA09157
:100470009400DA0ADD202AF4AFEFC094D094CA1AAF
:10048000DA0A20929500A8E0A210A0E0CA14DA06C9
:1004900018F4A1E0A093950040939300509394002A
:1004A000409191005091920040938F0050939000A2
:1004B00042E097C0A09165004A1BA09166005A0BCC
:1004C00094FD82C093FD80C092FD7CC086FF03C076
:1004D000D52EC42E0CC05695479591FD73C05695E8
:1004E000479590FD6FC0D52EC42ED694C79461FD5C
:1004F00019C0AC2DAC51AD2DA24008F005C0DD20D7
:1005000089F4AC2DA85C70F4A0916700A395AA2390
:1005100011F0A0936700AA3008F471C020929600F1
:1005200081606DC0A0916700AA2319F0AA95A093DD
:100530006700A22C5091BA0097FD06C0A090C80099
:10054000533011F4A090D000AAEFAA0EA22DA21D44
:10055000CA18DA0A4FB74170533049F4442321F0E6
:1005600087FD05C0806803C087FF01C08F774423E3
:1005700059F0533031F4AFEFC094D094CA1ADA0A6C
:1005800003C040E050E020C0533049F4CC0CDD1CE7
:10059000AAE0CA1AD20818F4A0E0CA2ED22CAFEFF3
:1005A000CA16D20418F04FEF50E00EC0A091AC0074
:1005B000CA9E412D000C441F50E008F012C04FEFBE
:1005C00050E00FC05695479594FF07C0552309F09A
:1005D0004FEFA42FA6954A0F521D4F3F520508F02A
:1005E0004FEF40939600816061FF09C0AFE1A09595
:1005F000A923AB299A2F8F7DBB2009F48062A8E143
:10060000A093680085FF03C0AAE0A093680061FD85
:1006100003C085FD01C08F7E85FD03C0A6E0A093C9
:100620006900F894A9B7A160A9BF84FF03C0A9B766
:10063000A062A9BF3FBE189511E00AC013E008C030
:100640001AE006C01EE104C014E602C018EC00C0A7
:1006500005E1BB27BA95F1F70A95D9F71A95C1F7C5
:1006600008952AE338E709C020E33CE806C02AE2FF
:1006700034EB03C025E238EC00C0B091AD00BA9570
:1006800009F4089512E0BB27AD9ABA95F1F7929A52
:10069000BA95F1F79298BA95F1F7AD98BA95F1F746
:1006A000123009F0AC9A123009F4949AB091AD006E
:1006B000BA95F1F7123009F0AC98123009F4949819
:1006C000B7E8BA95F1F71A95F1F6022FB22FBA955D
:1006D000F1F70A95D9F73A9581F6AD9A0895221B5C
:1006E00039E0001F3A9509F40895221F211B18F4E0
:1006F000210F8894F6CF0894F4CF622C722CB0E0CE
:100700008894B395221F331FE0F737952795889477
:10071000912E802E020B130B10F4192D082D10F4BE
:10072000889401C00894661C771CBA9571F7172D40
:10073000062D0895322D11232AF43A95009510952F
:10074000031B130BF894029F712C002D129F912C08
:10075000802C7894780C172D921C292DB4E06B2EE8
:100760002695179507956A94D9F7332321F00095BC
:100770001095031B130B0895089510917B00169597
:1007800000917A000795B0917E00B01B0B2FB091BD
:100790007F00B10B1B2F28F40038BFEF1B0740F080
:1007A00009C00F37120508F405C00FE710E002C0BA
:1007B00000E81FEF009383001093840008950091D8
:1007C0008300B09180000B0F10918400B0918100E4
:1007D0001B1F20E03091840033230AF42A95B09146
:1007E00082002B1F1AF4203F40F00AC02F3008F47B
:1007F00007C00FEF1FEF2FE003C000E010E020EF75
:1008000030916300B0919B003B1718F4323030F008
:1008100009C0B0918400BB235AF004C0B091840099
:10082000BB2332F400938000109381002093820058
:1008300008952091D70000918300000F109184004B
:10084000111F78DF11232AF40038BFEF1B0740F097
:1008500009C00F37120508F405C00FE710E002C009
:1008600000E81FEF002352F0B0916200B01B0B2F85
:1008700018F0013008F00AC001E008C000950F5FD1
:10088000B09162000B0F08F001C00FEF00938500DC
:1008900008952091D80000918100109182004ADFD4
:1008A00011232AF40130BFEF1B0740F009C00F3FAE
:1008B000120508F405C00FEF10E002C001E01FEFC1
:1008C000112352F0B0918500B01B0B2F18F00130AE
:1008D00008F00AC001E008C000950F5FB0918500E4
:1008E0000B0F08F001C00FEF0093630008950FEFA6
:1008F00071FD1EC0B091D300BB23D1F0B0917B003D
:10090000BB23B1F00FEF10917B00E9DEF894B091BA
:10091000730072FDB5E00B9F112D002D789411230B
:1009200009F00FEFB0919E000B1710F400919E009C
:1009300000939D00089500917A0010917B0000546F
:100940001140B0919D0010F4BA9501C0B39511F01B
:10095000B0939D00089500C008952091B500B6B1F0
:10096000B6FDFBCF04B115B1B6B1BF77B6B9B09142
:10097000AA00B395B093AA00B83060F12092AA0003
:10098000B091D200BB2321F1112329F0B091AB002B
:10099000BF3F61F009C0B091AB000B1739F020F4F4
:1009A000BB2321F0BA9502C0B395E1F300919B00FF
:1009B000B093AB00B03050F400ECB03038F400E845
:1009C000B03020F400E4B03008F400E000939B0065
:1009D0007F7E0895B0919B00B39511F0B0939B007A
:1009E000B091AA00B73009F47061089502E3F89459
:1009F000B091D9000B9F012D000C001F7894B0918D
:100A00009B000B1710F000919B0000936100009376
:100A10006300502E0093640000939E00089520927E
:100A20007A00B0EFB0937B000895F8940CB51DB533
:100A30002091740078943091750060907600009356
:100A4000750010937600031B160971FD03C077FD36
:100A500080C028C070907700209377002709222358
:100A600019F00FEF1FEF0EC0809078009090790082
:100A700030937800609279000091750010917600B3
:100A80000819190920917A0030917B003695279535
:100A9000020F131F10F40FEF1FEF00937A00109353
:100AA0007B002BC020917A0030917B003901B4E0AB
:100AB0008B2EB2E09B2E343040F08A949A943830DA
:100AC00020F072FD02C08A949A94769467948A9476
:100AD000E1F726193709992021F0169507959A9480
:100AE000E1F7200F311F20937A0030937B0028F428
:100AF0003FEF30937A0030937B00323008F4706817
:100B000071FF02C0B3E00DC0B091C400009171004C
:100B1000023838F0B395003A08F0B395B63008F0D3
:100B2000B5E09B2EB4E08B2E10917B0000917A00F3
:100B300024E0169507952A95E1F70819120928F07F
:100B4000B02FB250B12FB20910F402E010E09801BA
:100B500026C020917A0030917B0039017694679409
:100B60006694669466942619320906950695200FB8
:100B7000321D20937A0030937B00323008F07F776B
:100B800004E0369527953695279526952695201BC2
:100B900010F0223008F422E089019090C40060FD3A
:100BA000FECFE0908B00F0908C006160B9B7B0612F
:100BB000B9BF380177FD41C07694679400938B00EC
:100BC00010938C00B92DB330E1F0B0FD04C0060DD8
:100BD000171D930106C0000F111F0250120922E0D9
:100BE00030E0B92DB33068F020938D0030938E0043
:100BF00000938700109388006092890070928A00A9
:100C00003AC000938D0010938E002093870030939C
:100C100088006092890070928A0071FF0DC0BFE069
:100C2000B0938D0020928E00B093890020928A00AC
:100C3000B0938B0020928C001EC0669400938B00B2
:100C4000B92DB33091F0B0FD03C0060D262D03C0C1
:100C5000000F025022E0B92DB33038F020938D0000
:100C6000009387006092890006C000938D00209356
:100C700087006092890000917C0002FD03500130E2
:100C800029F495FD0AC0B6E0B7B909C0023019F4DD
:100C9000B7E0B7B904C095FDF6CFB0E0B7B90091A1
:100CA000A200000F10F4BBE60B270093A20060FD2A
:100CB000FECFB2E0B0936E006160B9B7B061B9BF6A
:100CC000B72FB670D1F020917A0030917B00369525
:100CD00027953695279571FF02C0B0E43B0FF89435
:100CE0000CB51DB5020F131F1BBD0ABD6160B0E13D
:100CF000B8BFB9B7B061B9BF789408956860209261
:100D00007D0020E066FD20E206C0686020927D0044
:100D100020E266FD20E001E011E077FD11C0B72F71
:100D2000B67009F0677F14E100917B00069509F425
:100D300003950F3008F00FE071FF02C004E114E1E9
:100D400060FD0FC0B0917D00BB2359F071FF06C05C
:100D5000B0916E00BA95B0936E0011F470624FC0FE
:100D6000ABDFB0B7B77FB0BFB8B1B0B7B860B0BF96
:100D7000B0917D00B395B0937D00B8B177FD06C00A
:100D8000B1E071FDB3E0BA95F1F7B8B1B072B21746
:100D900009F02AC071FF05C00395011708F00A95F4
:100DA000CFCF63FD05C00395011708F0B4CFC8CFBE
:100DB000677FF8943CB56DB470907A00B0917B0079
:100DC000770CBB1F08F4BFEF770CBB1F08F4BFEF15
:100DD000370D6B1E6BBC3ABD6160B0E1B8BFB9B7EF
:100DE000B061B9BF789497CFB0916D00B13008F47D
:100DF00092CF63FD90CF0A9509F0A2CF7F7D20911D
:100E00008D0030918E00F894B0E1B8BF0CB51DB5DF
:100E1000020F131F1BBD0ABDE0908700F0908800F1
:100E20006160B9B7B061B9BF7894B72FB67039F0C7
:100E3000B0916D0072FFB395B0936D0009C075FF5E
:100E400007C066FD05C063FD03C0BF91BF91FAC432
:100E5000089500E063FF01C001E0F8941091710073
:100E6000B7E01B9F212D102D7894200F2695179504
:100E7000269517952695179510937100183718F435
:100E8000B8E7B093710000917100B09172000B1738
:100E900020F06061AC989298949860FDFECFE0904D
:100EA0008900F0908A006160B9B7B061B9BF089558
:100EB000B2E095FD0AC0F894B0937C00AD9A959885
:100EC00062FF01C0949A7894F4C0F894B0937C00C7
:100ED000AD9A939862FF01C0AC9A7894EAC0B3E0EF
:100EE00082FF24C095FD11C002E0F894B0937C000D
:100EF000E0E8F0E00093B1009498939A62FF02C09A
:100F0000929A01C0AD987894D4C002E0F894B0935E
:100F10007C00E0E8F0E00093B100AC98959A62FFA5
:100F200002C0929A01C0AD987894C3C095FD0BC0E1
:100F3000F894B0937C00EAE6F0E0949862FF01C078
:100F4000929A7894B6C0F894B0937C00EAE6F0E008
:100F5000AC9862FF01C0929A7894ABC0B4E095FD62
:100F60000AC0F894B0937C00959A939862FF01C0F0
:100F7000929A78949EC0F894B0937C00939A959836
:100F800062FF01C0929A789494C0B5E082FF24C0B9
:100F900095FD11C001E0F894B0937C00E6E7F0E025
:100FA0000093B1009298AD9A62FF02C0AC9A01C062
:100FB000959878947EC004E0F894B0937C00EAE8B9
:100FC000F0E00093B1009298AD9A62FF02C0949A4B
:100FD00001C0939878946DC095FD0BC0F894B093C0
:100FE0007C00E4E6F0E0929862FF01C0AC9A78944D
:100FF00060C0F894B0937C00E0E7F0E0929862FF64
:1010000001C0949A789455C0B6E095FD0AC0F89452
:10101000B0937C00939AAD9862FF01C0AC9A78942B
:1010200048C0F894B0937C00959AAD9862FF01C0D7
:10103000949A78943EC0B1E082FF24C095FD11C01F
:1010400004E0F894B0937C00EAE8F0E00093B1008B
:10105000AC98959A62FF02C0949A01C093987894D4
:1010600028C001E0F894B0937C00E6E7F0E000933C
:10107000B1009498939A62FF02C0AC9A01C095980F
:10108000789417C095FD0BC0F894B0937C00E0E70E
:10109000F0E0AC9862FF01C0949A78940AC0F8948A
:1010A000B0937C00E4E6F0E0949862FF01C0AC9A53
:1010B00078946F7E089523E630E0F9012092B10024
:1010C000AC9892989498959AAD9A939A6B7F08955C
:1010D000A2EBB0E00FEF0D930D930D930D9303E092
:1010E0000D9304E00D930BE00D9303E00D9301E0ED
:1010F0000D9301E00D93AEEBB0E001E00D930FEF27
:101100000D930D930D930D930D9303E00D930FEF3E
:101110000D930FEF0D930D9305E20D9300ED0D93DD
:101120000AEF0D930AEF0D9304E00D930FEF0D936B
:1011300001E00D9300E00D930AE70D930FEF0D937F
:1011400000E00D9301E00D9300E00D9303E00D939B
:1011500000E00D9308952091B9008B7F233009F4AE
:101160008460B091BA00B33019F09F7DB1FD9062F8
:101170009F7BB091BB00B1FD9064223011F088607C
:1011800001C0877F08950A95E00FF21DB49108957C
:10119000ECE1F0E00091B200F6DFB093D700ECE1B3
:1011A000F0E00091B300EFDFB093D800EAE2F0E0A6
:1011B0000091B800E8DFB093D9000091B800023088
:1011C00008F402E000937300B091CE000FEFB2304C
:1011D00009F400EAB33009F402E800937200E8E38E
:1011E000F0E00091D500CFDFB093A00008950895FE
:1011F0002091C8003091C900B091BA00B33009F411
:101200003E5097FF02C020E03FEFB32FB21B6B2E82
:10121000B25810F4B2E86B2E00E00395609EB12D39
:10122000BD57D8F30093AC0008959068E1DF0ADA67
:1012300009DA20E030E0B0E16B2E00DAB0919600E0
:101240002B0F321D6A94C9F7B4E036952795BA95ED
:10125000E1F7822E9F77CCDF0895F894E3E0F0E089
:10126000B9E0B7BFB491B078C1F3F894A895B1B51F
:10127000B861B1BDB0E0B1BDB4E0BEBFBFE5BDBFB8
:101280001ADFB0E0B8BBB0E1B7BBB0E2B5BBB0E3CA
:10129000B4BBB8E2B2BBBCE3B1BB2224A0E0B0E077
:1012A0002D92AA31E9F7A0E6B0E00FEF2D920A9552
:1012B000E9F7B1E0B093A2000BDFFCD2B6B1B460A5
:1012C000B6B90091CA000093AD00B1E0B0936A00D6
:1012D000F894BCD9C6D9B6D9C7D9B4D9C8D9B2D966
:1012E00070D3B4D9B3D9B0D9F8940AEF1AEFA6B332
:1012F00096FDA095A0FF1FC01A95C9F70A95B1F7F2
:10130000E0E0FCE1B591B43E39F4B591B03E21F492
:10131000B591BF3F09F40CC0E0E0F395F395B591AA
:10132000B83F49F4B591B43931F4B591BA3A19F4EA
:10133000EE27F69509940FDF2BDF59DF59DF009177
:10134000CA000093AD00B7DEB2E0B3BFB2E0BEBDED
:10135000B2E0B5BDB1E5B8BFB9BFB0B7B77FB0BFF8
:10136000B8B1B0B7B860B0BF67D97894F4DA20925A
:101370007000BEB5B06496FDBF7BBEBDB9B7B062AC
:10138000B9BFBB27B062B8BF8D7F60D9626033E060
:101390002CE0B0919500BB2321F42CE03A9509F4A0
:1013A000A3CF50D980FFA0CF8E7FB0919600B230EE
:1013B00078F3B92FBF710091980000939700B09314
:1013C0009800B01729F72A9521F76D7FBEB5B06454
:1013D00096FDBF7BBEBDBB27B062B8BF8D7FB0910D
:1013E000D400BB2321F48062B92FB0709B2F8F7B78
:1013F0002092670029D985FF05C0B0916700BA30F7
:1014000008F080641BD902E085FF01C000E0B091C4
:101410009600B017B8F3F89424D923D922D9789438
:1014200015D920928600B091BA00B33009F47EC07D
:1014300005D9B091BE00B13008F478C0B0916A000F
:10144000B13008F473C085FD18C0B0919600BF3F5D
:1014500008F46CC0F8940ED97894F6D8B091960040
:10146000B130C0F7F894FDD8EBD8FBD87894ECD81D
:10147000B0919600BF3FB0F3D6C2B8E09B2E906803
:10148000F894B6DE7894E0D8F8949F77B1DE809037
:101490009600B0919600BF37789408F44FC0CCD82E
:1014A000F894E8D878949A9451F7BFDEB82DB550E7
:1014B000B093C900CBD8F89489D27894BAE09B2E27
:1014C0009068F89495DE7894BFD8F8949F7790DE72
:1014D00080909600B0919600BF37789478F7ACD89A
:1014E000F894BFD8ADD8BDD878949A9449F79DDECA
:1014F000B82DBB5FB093C8000B2F1091C9001258D4
:1015000010F0100B20F4B2E80B0F0093C9009ED826
:10151000F894FDD16AD2789497D8F89469DE7894DB
:10152000B0919600BF3F08F48ECF7DC20091960027
:10153000B09186000B1710F00093860085D801E06B
:10154000B091BA00B35009F405E0B0919600B0171D
:1015500008F069CFF8948ED88DD88CD8789476D846
:1015600020926A0020926B0020926C00B0916B0078
:10157000B395B0936B00BF3F71F5B0916C00B3951C
:10158000B0936C00B091CC0009E1BA9559F002E338
:10159000BA9541F00DE7BA9529F00AEFBA9511F026
:1015A00020926C00B0916C00B017A8F084DD44D894
:1015B000B0916C00BA95B0936C0020926B00B09122
:1015C000CB00B093AD00F89455D87894B091CA0090
:1015D000B093AD0039D834D8B0916800BB2319F46A
:1015E00085FF01C081CE01E085FD01C006E0B0911C
:1015F0009600B01708F4BACFB091BA00B35009F012
:1016000023D8B0916800BB2309F46ECEF89453DD63
:10161000209261002092620020926300522C20925E
:1016200064002092A1007894B091B700BB0FB093F2
:101630009F0020927E0020927F00209280002092C6
:101640008100209282002092AA0060E070E0209247
:101650007100B8E0B093AA007061EED7B2E074FDFB
:10166000B2E0B7B9B6B1B068B064B6B9B6B1B6FD5C
:10167000FDCF04B115B1B6B1BF77B6B9112309F0EA
:101680000FEF0093AB0069D9B8E0B093AA00706186
:1016900062DDF894BFEFB0939B00A8D9B0916100D0
:1016A000B0939B00B0939C00B0939D007894B1E000
:1016B000B0936100B09363005B2EB0936400B0936D
:1016C000A400B0919A00B093A300B091BA00B330D7
:1016D00019F49F7D87FD90627160726020926D00A9
:1016E00093DCA9DC9CD9A1D99AD99FD998D90DDBD3
:1016F00043D8AFDBDDDB99D901DB65FD3ED877FF51
:10170000F6D877FD18D9A5DBEADB8FD9FEDA65FDBF
:1017100056D89FDB23DC89D9F1DA65FD8AD899DBBD
:1017200034DC83D9F2DA65FDB4D893DB6DDC7DD986
:10173000E5DAB2E074FDB2E0B7B9B6B1B068B06452
:10174000B6B987DB78DC71D908D971FF21C0B091B7
:101750009E00B0939B00B0939C00B0919A00B09310
:10176000A300B1E0B093A40018E12CE0B0916D00AB
:10177000B11740F07D7F746020936F00BFEFB0938E
:101780009B0006C0B0919600B13008F0B0CF64C0A5
:1017900072FF15C066FD13C0B0916F00BA9519F4C1
:1017A0007B7F7860A4CFB0936F00B0919600B1308A
:1017B00008F09DCFB091BA00B33009F04DC020922F
:1017C0007000B091990002E81091D600112309F041
:1017D00003E0B01708F040C085FF04C0B091680076
:1017E000BB23D1F1B091BA00B33081F495FD03C0B1
:1017F00087FD04C00BC087FF01C008C066FD06C09E
:101800006064B0919E00B0939B0086CF00EF66FFAE
:1018100005C0B0919E00B0939B0000E2B0917B00A8
:10182000B01708F464CF66FF17C06F7B9F7D87FDFC
:1018300090627460B2E1B0936F00B0919E00B0937B
:101840009B0055CFB0917000B395B0937000B091EC
:101850009600BB2309F002C020927000F8942BDCA4
:101860008090B900B2E0B093B90075DC8092B90005
:10187000209261002092620020926300522C2092FC
:10188000640020929F0060E070E07894DDD613DC65
:101890000091D600002319F0AC9A929A949AB6B1AE
:1018A000B460B6B985FF05C0B0917000B43008F0DF
:1018B0001BCD58CEEDE0F0E023D00A3509F01BC077
:1018C000EEE0F0E01DD0053A09F015C03AE0A2EBD9
:1018D000B0E0E3E0F0E014D00D9331963A95D9F7FB
:1018E00039E1AEEBB0E0EFE0F0E00AD00D933196D5
:1018F0003A95D9F702C0ECDB0AD0E8E2F0E00895AF
:10190000E199FECFEEBBFFBBE09A0DB308951ED068
:101910003AE0A2EBB0E0E3E0F0E00D910FD03196B9
:101920003A95D9F739E1AEEBB0E0EFE0F0E00D9198
:1019300005D031963A95D9F712D00895E199FECFA6
:101940000DBBEEBBFFBBE29AE19A0895EDE0F0E03B
:101950000FEFF4DFEEE0F0E00FEFF0DF0895EDE0E1
:10196000F0E00AE5EBDFEEE0F0E005EAE7DF0895FE
:101970003091AE000091AF00313011F40093B60009
:10198000323011F40093B700333011F40093B800F3
:10199000343011F40093C400353011F40093B900D1
:1019A000363011F40093D500373011F40093CE0097
:1019B000383011F40093BA00393011F40093BB00B1
:1019C000089525E043D62A95E9F708954AD64CD6DE
:1019D0004ED650D635D645D647D649D64BD630D634
:1019E00040D642D644D646D6089544D640D63CD6B4
:1019F00038D626D63FD63BD637D633D621D63AD69A
:101A000036D632D62ED608958090AE009090AF0094
:101A100028D627D626D614D68A94D1F72BD610D618
:101A20009A94E1F70895F894D1DF7894CADFC9DF7A
:101A3000B1E0B093AE00B1E0B093AF002092B0003F
:101A4000F894E2DF7894B5E06B2E70909600FED5A6
:101A5000B09196007B16C9F7B13018F0BF3F40F146
:101A600007C086DFF89453DFB1DFB8E0B1BDA9DF6E
:101A70006A9459F7B091B000B395B093B000B33009
:101A800008F4DECF9EDFB091AF00B395B093AF0006
:101A9000F894B091AE00BA95EEE3F0E0EB0FF21DD2
:101AA000049178940395B091AF00B01708F4C6CFB5
:101AB00088DF87DFB091AE00B395B093AE00B091F0
:101AC000AE00BA3008F4B7CF03DBF89420DFB8E0FB
:061AD000B1BD77DFC2CBBF
:00000001FF
